:100000000C9430050C9477050C9477050C947705C7
:100010000C9477050C9477050C9477050C94770570
:100020000C9477050C9477050C94930C0C94650D47
:100030000C94D01B0C9477050C9477050C947705E1
:100040000C9477050C9477050C9477050C94770540
:100050000C9477050C94701C0C9477050C94770520
:100060000C9477050C9477050C9477050C94770520
:100070000C9477050C9477050C9477050C94770510
:100080000C9477050C9477050C9477050C94770500
:100090000C9477050C9477050C9477050C947705F0
:1000A0000C9477050C9477050C947705D20DF40D1C
:1000B000E20EF40DE20E390E5C0EE20EB10EC40E2D
:1000C000D911D911071207126412A212BB14BB1462
:1000D000BB12BB14BC13BC138F14BB14BB14A614EB
:1000E0008080352B787939808080210877060780D9
:1000F0008080201A7A1B168080801E802980808054
:100100008080808080808080808022158019098096
:1001100080801F147B1D0480808023172C050A809B
:100120008080260C00360E808080251876100D8089
:100130008080241C80110B80808027127E370F80E6
:1001400080802A804F7D2880808074305152328098
:1001500080802D137C38338080802E2F5075348022
:100160004B6579626F6172642073746172742E0AD8
:100170000055534220636F6E666967757265642E21
:100180000A000D0A696E69740A005B445D005B43F6
:100190005D001203480048004B00420020006D0043
:1001A0006F00640000000E0374002E006D002E002E
:1001B0006B002E0000000403090409028D000501F4
:1001C00000A032090400000103010100092111010E
:1001D00000012240000705810308000A090401000C
:1001E0000103010200092111010001224D00070550
:1001F000820308000A09040200010300000009212B
:10020000110100012236000705830308000A0904D2
:100210000300020300000009211101000122220055
:1002200007058403200001070504032000010904D9
:10023000040001030000000921110100012239001E
:10024000070585032000011201100100000008EDE0
:10025000FEFECA04010102000105010906A1010513
:100260000719E029E71500250195087501810205A8
:1002700008190129059505750191029501750391EC
:10028000010507190029F71500250195F875018169
:1002900002C00631FF0974A1010975150026FF008F
:1002A0009520750881020976150026FF00952075B6
:1002B000089102C005010980A1018502168100266E
:1002C000B7001A81002AB700751095018100C0059A
:1002D0000C0901A1018503160100269C021A0100E8
:1002E0002A9C02751095018100C005010902A10137
:1002F0000901A10005091901290515002501950528
:1003000075018102950175038101050109300931EB
:100310001581257F95027508810609381581257F8D
:10032000950175088106050C0A38021581257F950F
:100330000175088106C0C005010906A1010507195C
:10034000E029E715002501950875018102950175E1
:100350000881010508190129059505750191029586
:1003600001750391010507190029FF150026FF00FB
:10037000950675088100C0636F6E73756D65723A7E
:1003800020253034580A0073797374656D3A20253E
:100390003034580A000A002530325820006B657945
:1003A000626F6172643A20004C45443A2025303235
:1003B000580A00253032583A202530386225730A11
:1003C00000722F632030313233343536370A0064FF
:1003D000656C5F6B65795F6269743A2063616E2753
:1003E000742064656C3A20253032580A00616464D8
:1003F0005F6B65795F6269743A2063616E27742070
:100400006164643A20253032580A004F6E65736883
:100410006F743A2074696D656F75740A00290A005B
:100420002575002F002575005D280025640020003B
:10043000256400200025640020002564007C002540
:10044000303258006D6F7573656B6579205B62742F
:100450006E7C782079207620685D287265702F6127
:10046000636C293A205B006D6B5F776865656C5F34
:1004700074696D655F746F5F6D6178203D202564E0
:100480000A006D6B5F776865656C5F6D61785F739F
:1004900070656564203D2025640A006D6B5F74699A
:1004A0006D655F746F5F6D6178203D2025640A0083
:1004B0006D6B5F6D61785F7370656564203D2025AD
:1004C000640A006D6B5F696E74657276616C203DC5
:1004D0002025640A006D6B5F64656C6179203D20A6
:1004E00025640A006D6B5F776865656C5F74696D84
:1004F000655F746F5F6D6178203D2025640A006D33
:100500006B5F776865656C5F6D61785F737065655B
:1005100064203D2025640A006D6B5F74696D655F22
:10052000746F5F6D6178203D2025640A006D6B5FFC
:100530006D61785F7370656564203D2025640A00F5
:100540006D6B5F696E74657276616C203D20256409
:100550000A006D6B5F64656C6179203D2025640A3B
:10056000000A00257500363A20776865656C5F746F
:10057000696D655F746F5F6D61783A20000A0025D0
:100580007500353A20776865656C5F6D61785F73DB
:10059000706565643A20000A00257500343A2074BD
:1005A000696D655F746F5F6D61783A20000A0025A0
:1005B0007500333A206D61785F73706565643A2029
:1005C000000A00257500323A20696E746572766102
:1005D0006C286D73293A20000A00257500313A20F5
:1005E00064656C6179282A31306D73293A20000ADC
:1005F000092D2056616C756573202D0A004D3E0053
:100600004D25643E20003F0073657420646566617B
:10061000756C740A00433E2000776865726520643B
:10062000656C74613A20637572736F723D25642C3A
:1006300020776865656C3D25640A5365652068749C
:1006400074703A2F2F656E2E77696B6970656469D7
:10065000612E6F72672F77696B692F4D6F757365A8
:100660005F6B6579730A000A092D204D6F757365FC
:100670006B6579202D0A4553432F713A09717569CD
:10068000740A313A0964656C6179282A31306D73D6
:10069000290A323A09696E74657276616C286D7345
:1006A000290A333A096D61785F73706565640A34AD
:1006B0003A0974696D655F746F5F6D61780A353AE8
:1006C00009776865656C5F6D61785F7370656564F7
:1006D0000A363A09776865656C5F74696D655F74A1
:1006E0006F5F6D61780A0A703A097072696E7420E2
:1006F00076616C7565730A643A0973657420646584
:100700006661756C74730A75703A092B310A646FEF
:10071000776E3A092D310A706775703A092B3130BE
:100720000A7067646F776E3A092D31300A0A737068
:10073000656564203D2064656C7461202A206D61CC
:10074000785F7370656564202A2028726570656122
:1007500074202F2074696D655F746F5F6D617829F7
:100760000A003F004D3E2000433E20004C25640A15
:10077000000A092D20436F6E736F6C65202D0A45AA
:1007800053432F713A09717569740A6D3A096D6F97
:100790007573656B65790A000A092D204D616769DB
:1007A00063202D0A643A0964656275670A783A091C
:1007B0006465627567206D61747269780A6B3A09C5
:1007C0006465627567206B6579626F6172640A6D3A
:1007D0003A096465627567206D6F7573650A763ACC
:1007E0000976657273696F6E0A733A09737461747E
:1007F00075730A633A09636F6E736F6C65206D6F72
:1008000064650A302D343A096C61796572302D3493
:10081000284631302D4634290A506175733A0962F1
:100820006F6F746C6F616465720A6E3A094E4B5259
:100830004F0A003F004E4B524F3A206F66660A0047
:100840004E4B524F3A206F6E0A0074696D65725FAD
:1008500072656164333228293A202530346C580A95
:10086000006B6579626F6172645F6E6B726F3A20C4
:1008700025580A006B6579626F6172645F69646C08
:10088000653A2025580A006B6579626F6172645F72
:1008900070726F746F636F6C3A2025580A00686F2E
:1008A00073745F6B6579626F6172645F6C656473AA
:1008B00028293A2025580A000A092D20537461740A
:1008C0007573202D0A004743433A20342E392E32C7
:1008D000204156522D4C4942433A20312E382E3079
:1008E00073766E204156525F415243483A206176FA
:1008F00072350A004F5054494F4E533A204C5546DA
:1009000041204D4F5553454B455920455854524170
:100910004B455920434F4E534F4C4520434F4D4D6F
:10092000414E44204E4B524F204B45594D41505F54
:1009300053454354494F4E20343039360A0042550E
:10094000494C443A20353732633236352D6469726A
:100950007479202831343A33313A3034204A616E88
:100960002032352032303137290A005649443A20A6
:1009700030784645454428742E6D2E6B2E29205024
:1009800049443A203078434146452848484B422064
:100990006D6F6429205645523A203078303130341A
:1009A0000A00444553433A20742E6D2E6B2E206B63
:1009B0006579626F617264206669726D77617265D4
:1009C00020666F722048484B42206D6F640A000A0F
:1009D000092D2056657273696F6E202D0A000A6D0D
:1009E0006F7573653A206F66660A000A6D6F7573DE
:1009F000653A206F6E0A000A6B6579626F617264F6
:100A00003A206F66660A000A6B6579626F617264EC
:100A10003A206F6E0A000A6D61747269783A206F2D
:100A200066660A000A6D61747269783A206F6E0A10
:100A3000000A64656275673A206F6E0A000A646591
:100A40006275673A206F66660A000A0A626F6F7401
:100A50006C6F616465722E2E2E2000433E200000D4
:100A600011241FBECFEFDAE0DEBFCDBF04B603FE18
:100A700027C08091220290912302A0912402B0917C
:100A800025028730904BA740B04BD1F41092220240
:100A900010922302109224021092250214BE84B7F1
:100AA000877F84BF0FB6F894A89580916000886115
:100AB00080936000109260000FBEE0E0F8E30995BB
:100AC00011E0A0E0B1E0E6EFF9E402C005900D927C
:100AD000A833B107D9F722E0A8E3B1E001C01D9225
:100AE000A232B207E1F70E94C1090C94F9240C94D8
:100AF0000000FF93EF93E0913801F09139013097B6
:100B000009F00995EF91FF910895FC0185918030DE
:100B100011F0EFDFFBCF0895FF27E0E230E247FF5F
:100B20000CC0419597FF09C0EDE2609570958095E6
:100B30009095611D711D811D911D27FF02C021959A
:100B400030E350E2AA27660F771F881F991FAA1F5C
:100B5000A41710F0A41B63955A95A9F7AA3008F0C2
:100B6000A95FA05DAF93F3956115710581059105AE
:100B700041F7ED3211F4EF93F395F21718F43F9328
:100B8000F395FBCF8F91B5DFFA95E1F70895E991E1
:100B9000F9918591803021F0853219F0AADFF9CFE3
:100BA000089520E0E89455915532C1F3503311F483
:100BB000689455915A3348F4505390F3220F022E03
:100BC000220F220F200D250FF4CF0EF421958991CD
:100BD0009991533619F3533729F1533559F1BC0123
:100BE00088279927E8945C3621F489919991689433
:100BF0005591543639F446EF7EF077FF0DC08FEFF4
:100C00009FEF0AC055374AE039F0583540E121F0EE
:100C1000523642E009F00895FF93EF937DDFEF91A4
:100C2000FF91B7CFFF93EF93FC0181918030B9F32F
:100C300060DFFBCFFF93EF9368DFF1CFDF93CF93BC
:100C4000CDB7DEB72596A3DFCF91DF9108958FEF63
:100C500084B980E485B957985F9A87B1806C87B969
:100C600088B1806C88B92E9A2F98EAE4F1E080E18F
:100C70008E0F11928E13FDCFEAE3F1E080E18E0F2B
:100C800011928E13FDCF8AE491E090935D018093E1
:100C90005C018AE391E090935B0180935A0108958F
:100CA000EF92FF920F931F93CF93DF9380915A019E
:100CB00090915B0120915C0130915D0130935B016B
:100CC00020935A0190935D0180935C01C0E0D0E0D5
:100CD00001E010E080E090E0FC2FF770EC2FE8706E
:100CE00025B1207C2F2BAC0133E0440F551F3A95E2
:100CF000E1F7242B25B928B12F73EE2311F02064DE
:100D000001C0206828B92AE12A95F1F700C0A09116
:100D10005A01B0915B01AC0FBD1F2C9130E0082E41
:100D200002C0359527950A94E2F720FD2F9AA5E396
:100D3000AA95F1F70000F6B42E98BAE1BA95F1F74A
:100D400000C040915C0150915D01BA016C0F7D1FA4
:100D50004F9B0BC09801082E01C0220F0A94EAF79E
:100D60002095DB013C91232309C0DB01EC90980125
:100D7000082E01C0220F0A94EAF72E292C9326B5DB
:100D80006F2D70E02F1518F026B530E004C026B5A1
:100D900030E021503F4F261B370B2630310558F0ED
:100DA000A0915A01B0915B01AC0FBD1F2C91DA01EB
:100DB000AC0FBD1F2C93BAE1BA95F1F700C02F9884
:100DC0002E9A20EA2A95F1F701968830910509F0CC
:100DD00087CFA0915C01B0915D01AC0FBD1FE09188
:100DE0005A01F0915B01EC0FFD1F9C9180819817D7
:100DF00051F00E940E1C60935E0170935F0180931E
:100E00006001909361012196C031D10509F062CF54
:100E100080911902853021F080911902811111C051
:100E200060915E0170915F0180916001909161011C
:100E30000E94441C613177428105910510F00E94A7
:100E40008F1B81E0DF91CF911F910F91FF90EF9069
:100E5000089520915C0130915D01F901E80FF11DC9
:100E60008081089508950895569A81FF02C05E9A80
:100E700008955E9808958091860108959FB7F8942B
:100E8000109265019FBF90911902943009F057C0EC
:100E90009091E9009F703091EC00232F217030FD7C
:100EA00020E8922B24E02093E9002091EB0020FF22
:100EB00043C02091EE0027FF3FC020916201222312
:100EC00021F02091E80025FF37C01092620126E052
:100ED0003091E80035FD15C030911902343061F5CC
:100EE0003091EB0035FD28C0215021F481E0809342
:100EF000620122C0EFE9FFE03197F1F700C0000086
:100F0000E7CF8093F1008091E80085FD0AC08091D1
:100F1000E80080FFFCCF8091E8008E778093E800A6
:100F200006C08FB7F89421E0209365018FBF9F70B2
:100F30009093E90080E008959F709093E9008FEF0F
:100F40000895CF93DF9300D01F92CDB7DEB79C01F9
:100F500080911902843019F593E099833B832A83A9
:100F60009093E9008FEF9091E800815095FD06C0C5
:100F700095ED9A95F1F700008111F5CF8091E80089
:100F800085FF0DC040E050E063E070E0CE010196C7
:100F90000E94830A8091E8008E778093E8000F908A
:100FA0000F900F90DF91CF910895CF93DF9300D0F2
:100FB0001F92CDB7DEB720911902243021F522E02F
:100FC00029839B838A8383E08093E9008FEF90914C
:100FD000E800815095FD06C095ED9A95F1F7000067
:100FE0008111F5CF8091E80085FF0DC040E050E011
:100FF00063E070E0CE0101960E94830A8091E800D0
:101000008E778093E8000F900F900F90DF91CF9133
:101010000895209119022430F1F422E02093E90090
:101020002FEF3091E800215035FD06C035ED3A959F
:10103000F1F700002111F5CF2091E80025FF0BC04A
:1010400040E050E065E070E00E94830A8091E80093
:101050008E778093E8000895CF93DF932091190253
:10106000243009F048C0EC0180910A018823E1F0A6
:1010700080910B018823C1F085E08093E9008FEF18
:101080009091E800815095FD06C095E19A95F1F7A1
:1010900000008111F5CF8091E80085FF2CC040E071
:1010A00050E060E270E017C081E08093E9008FEFCC
:1010B0009091E800815095FD06C095ED9A95F1F765
:1010C00000008111F5CF8091E80085FF14C040E059
:1010D00050E068E070E0CE010E94830A8091E80051
:1010E0008E778093E80080E2FE01A6E6B1E00190F1
:1010F0000D928A95E1F7DF91CF9108958EE891E006
:101100000E94850580911802811109C00E94180C67
:101110000E94750C8091E20084608093E200089543
:101120008AE891E00E9485051092180208950895BA
:10113000209163012F5F822F62E30E94BF249923D5
:1011400019F0209363010895109263018091650165
:10115000882371F180911902843041F58091E90072
:101160008F702091EC00922F917020FD90E8892BD8
:1011700094E09093E9009091EB0090FF14C090915F
:10118000EE0097FF10C09091E80095FF03C0109209
:10119000F100F9CF9091E80090FF05C09091E80030
:1011A0009E779093E8008F708093E900109265011C
:1011B000089542E061EC81E00E94920B42E061EC14
:1011C00082E00E94920B42E061EC83E00E94920B6D
:1011D00042E261EC84E00E94920B42E261EC85E025
:1011E0000C94920B80911B02833009F455C030F4AB
:1011F000813071F0823009F48EC008958A3009F48C
:101200007AC08B3009F460C0893009F09CC020C0DE
:1012100080911A02813A09F096C08091E800877F98
:101220008093E80080911E0290911F02892B21F487
:1012300060E286E691E003C060E080E090E070E06C
:101240000E94CE0A8091E8008B778093E800089591
:1012500080911A02813209F076C080911E0290912D
:101260001F02009719F0049709F06DC08091E80003
:10127000877F8093E8008091E80082FD05C080911F
:1012800019028111F8CF5FC08091F100809386012F
:101290008091E8008B7753C080911A02813A09F05F
:1012A00052C080911E0290911F02892B09F04BC001
:1012B0008091E800877F8093E8008091E80080FFBC
:1012C000FCCF80910A0136C080911A028132D9F593
:1012D00080911E0290911F02892BA9F58091E80050
:1012E000877F8093E8000E94C70B80911C02809347
:1012F0000A010C94DD1480911A02813221F580914B
:10130000E800877F8093E8000E94C70B80911D0250
:1013100080938701089580911A02813AA1F4809107
:10132000E800877F8093E8008091E80080FFFCCF91
:10133000809187018093F1008091E8008E778093FF
:10134000E8000C94C70B08950895089580918601D4
:10135000809364011092860180E00E9434070E940D
:1013600080100C94DD140C94A6090E948F1B8091B0
:101370001702882329F00E94B81B81110C946D0A72
:10138000089584B7877F84BF0FB6F894A89580919D
:101390006000886180936000109260000FBE90E052
:1013A00080E80FB6F89480936100909361000FBEBF
:1013B0008EE397E00E94601B82E891E00E94850521
:1013C0000E94A4090E94BB0F0E94180C0E94750C79
:1013D0008091E20084608093E20078948091190209
:1013E0008430E1F781E791E00E9485050E94BD0FFE
:1013F00080E091E00E94FA0E80E691E00E9485056F
:101400000E94A50980911902853019F40E94B5093E
:10141000F9CF0E94C10FF6CF0E94CC1B80916401CE
:101420008093860108950C940C0A292F33272330CA
:101430003105C9F064F42130310581F022303105E5
:1014400009F043C08DE890E02AEB31E042C0213240
:101450003105F1F02232310541F137C082E190E0EF
:1014600027E432E036C099278130910541F082307F
:10147000910541F0892B49F5E6EBF1E005C0E6EA7C
:10148000F1E002C0E2E9F1E0849190E09F0121C027
:101490006530D8F4E62FF0E0EE0FFF1FED5DFE4F54
:1014A0002081318189E090E014C0653070F470E0F3
:1014B000FB01EE0FFF1FE75EFE4F20813181FB0134
:1014C000EC5EFE4F808190E004C080E090E020E080
:1014D00030E0FA0131832083089580E189BD82E103
:1014E00089BD09B400FEFDCF8091D8008F7D809327
:1014F000D8008091E00082608093E0008091E0005D
:1015000081FDFCCF0895CF92DF92EF92FF920F936F
:101510001F93CF93DF93EC018B016A010E94E60BCE
:10152000811133C0C114D10439F0F6018081918159
:10153000081B190BC80FD91FE12CF12C011511053F
:1015400019F18091E80085FD16C08091E8008E7742
:101550008093E800C114D10449F0F60180819181A3
:10156000E80EF91EF182E08285E00FC00E94E60BD2
:10157000882321F30AC089918093F1000150110959
:10158000FFEFEF1AFF0ADACF80E0DF91CF911F91D2
:101590000F91FF90EF90DF90CF900895209120025F
:1015A000309121022617370748F06115710539F48B
:1015B0002091E8002E772093E80001C0B90140E0B7
:1015C00061157105A9F120911902222309F443C084
:1015D000253009F442C02091E80023FD40C020914D
:1015E000E80022FD32C02091E80020FFE9CF4091C1
:1015F000F3002091F20030E0342BFC01CF016115A3
:10160000710559F02830310540F481918093F10043
:10161000615071092F5F3F4FF1CF41E02830310514
:1016200009F040E02091E8002E772093E800C8CF31
:101630004111C9CF0AC080911902882361F0853019
:1016400061F08091E80083FD0AC08091E80082FF8C
:10165000F2CF80E0089582E0089583E0089581E06C
:10166000089520912002309121022617370748F073
:101670006115710539F42091E8002E772093E80078
:1016800001C0B901FC0120E06115710591F1809163
:101690001902882309F440C0853009F43FC08091C5
:1016A000E80083FD3DC08091E80082FD2FC080915D
:1016B000E80080FFE9CF2091F3008091F20090E0F4
:1016C000922B6115710559F08830910540F42491F1
:1016D0002093F1003196615071090196F2CF21E01B
:1016E000089709F020E08091E8008E778093E80069
:1016F000CBCF2111CCCF0AC080911902882361F091
:10170000853061F08091E80083FD0AC08091E80097
:1017100082FFF2CF80E0089582E0089583E008958B
:1017200081E00895982F973058F59093E900981725
:1017300039F07091EC002091ED005091F00003C061
:10174000242F762F50E021FF19C03091EB003E7F0F
:101750003093EB003091ED003D7F3093ED00309100
:10176000EB0031603093EB007093EC002093ED00C0
:101770005093F0002091EE0027FF07C09F5FD3CF6A
:101780008F708093E90081E0089580E00895809152
:101790001A0287FF11C08091E80082FD05C0809188
:1017A00019028111F8CF11C08091E8008B770BC02E
:1017B00080911902882349F08091E80080FFF8CFDA
:1017C0008091E8008E778093E80008952091E400EE
:1017D0003091E50095E64091EC00842F817040FF48
:1017E00022C08091E80080FD1CC0809119028823EE
:1017F00091F0853091F08091EB0085FD10C0409113
:10180000E4005091E5004217530729F39A019150E3
:1018100011F784E0089582E0089583E0089581E05F
:10182000089580E008954091E80042FFDECF0895DA
:101830000E94860C0E948E0CE0EEF0E080818160B8
:101840008083E8EDF0E080818F77808319BCA7ED7D
:10185000B0E08C918E7F8C9380818F7E80831092FC
:10186000180208950F931F93CF93DF930E94860C65
:101870000E948E0CC8EDD0E088818F7788838881A4
:101880008068888388818F7D888319BC10921902B3
:1018900010921502109217021092160200EE10E03C
:1018A000F80180818B7F808388818160888342E01A
:1018B00060E080E00E94920BE1EEF0E080818E7F9C
:1018C0008083E2EEF0E080818160808380818860A7
:1018D0008083F80180818E7F808388818061888306
:1018E000DF91CF911F910F910895E8EDF0E0808195
:1018F0008F7E8083E7EDF0E080818160808384E0EB
:1019000082BF81E0809318020C94320CE8EDF0E085
:1019100080818E7F80831092E20008951092DA0019
:101920001092E10008951F920F920FB60F921124AA
:101930002F933F934F935F936F937F938F939F93D7
:10194000AF93BF93EF93FF938091E10082FF0BC0B1
:101950008091E20082FF07C08091E1008B7F80933D
:10196000E1000E9498088091DA0080FF1FC08091FA
:10197000D80080FF1BC08091DA008E7F8093DA0050
:101980008091D90080FF0DC080E189BD82E189BDD1
:1019900009B400FEFDCF81E0809319020E947E0809
:1019A00005C019BC109219020E9490088091E100B4
:1019B00080FF19C08091E20080FF15C08091E20095
:1019C0008E7F8093E2008091E20080618093E2004C
:1019D0008091D80080628093D80019BC85E0809304
:1019E00019020E94B3098091E10084FF30C0809108
:1019F000E20084FF2CC080E189BD82E189BD09B489
:101A000000FEFDCF8091D8008F7D8093D80080911B
:101A1000E1008F7E8093E1008091E2008F7E8093D1
:101A2000E2008091E20081608093E20080911502E3
:101A3000882311F084E007C08091E30087FD02C095
:101A400081E001C083E0809319020E94130A809113
:101A5000E10083FF29C08091E20083FF25C08091CF
:101A6000E100877F8093E10082E080931902109269
:101A700015028091E1008E7F8093E1008091E20069
:101A80008E7F8093E2008091E20080618093E2008B
:101A900042E060E080E00E94920B8091F00088605C
:101AA0008093F0000E949708FF91EF91BF91AF9152
:101AB0009F918F917F916F915F914F913F912F9166
:101AC0000F900FBE0F901F9018951F920F920FB698
:101AD0000F9211242F933F934F935F936F937F93B4
:101AE0008F939F93AF93BF93CF93DF93EF93FF9326
:101AF000C091E900CF708091EC00D82FD17080FDAB
:101B0000D0E81092E9008091F000877F8093F00088
:101B100078940E94A90D1092E9008091F0008860ED
:101B20008093F000CD2BCF70C093E900FF91EF912F
:101B3000DF91CF91BF91AF919F918F917F916F91E5
:101B40005F914F913F912F910F900FBE0F901F907B
:101B500018951F93CF93DF93CDB7DEB7AA970FB633
:101B6000F894DEBF0FBECDBFEAE1F2E088E08E0F51
:101B70009091F10091938E13FBCF0E94F208809117
:101B8000E80083FF1FC180911A0290911B02492F28
:101B900050E04A30510508F015C1FA01EA5AFF4FEA
:101BA0000C94DF24803881F0823809F00BC18091D9
:101BB0001E028F708093E9008091EB0085FB8827DF
:101BC00080F91092E90006C08091160290911702E8
:101BD000911182609091E800977F9093E800809344
:101BE000F1001092F100C8C0282F2D7F09F0EAC043
:101BF000882319F0823061F0E5C080911C028130A9
:101C000009F0E0C0933009F080E0809317022BC008
:101C100080911C02811127C080911E028F7009F4EF
:101C2000D1C08093E9002091EB0020FF1CC09330CD
:101C300021F48091EB00806214C09091EB009061E0
:101C40009093EB0021E030E0A90102C0440F551F42
:101C50008A95E2F74093EA001092EA008091EB0047
:101C600088608093EB001092E9008091E800877F04
:101C700086C08111A7C010911C021F778091E300DC
:101C80008078812B8093E3008091E800877F8093A8
:101C9000E8000E94C70B8091E80080FFFCCF809194
:101CA000E30080688093E300111102C082E001C06C
:101CB00083E08093190286C08058823008F082C089
:101CC00080911C0290911D028C3D53E0950779F59F
:101CD00083E08A838AE289834FB7F894DE01139602
:101CE00020E03EE051E2E32FF0E050935700E49112
:101CF00020FF03C0E295EF703F5FEF708E2F90E002
:101D0000EA3010F0C79601C0C0968D939D932F5F67
:101D1000243149F74FBF8091E800877F8093E80026
:101D20006AE270E0CE0101960E94CE0A14C0AE01B4
:101D30004F5F5F4F60911E020E94150ABC01892B04
:101D400009F440C09091E800977F9093E800898162
:101D50009A810E94310B8091E8008B778093E80094
:101D600031C0803879F58091E800877F8093E80062
:101D7000809115028093F1008091E8008E77809326
:101D8000E8000E94C70B1EC081111CC090911C026C
:101D90009230C0F48091E800877F8093E8009093B0
:101DA00015020E94C70B80911502811106C0809117
:101DB000E30087FD02C081E001C084E08093190246
:101DC0000E94D9088091E80083FF0AC08091E80052
:101DD000877F8093E8008091EB0080628093EB0026
:101DE000AA960FB6F894DEBF0FBECDBFDF91CF919C
:101DF0001F91089590938D0180938C010895E09137
:101E00008C01F0918D01309721F00190F081E02D4F
:101E1000099480E00895EF92FF920F931F93CF9360
:101E2000DF93E0918C01F0918D013097B1F18C013D
:101E30000280F381E02D09958091040282FF2DC07C
:101E400080FF04C08DE993E00E948505E80110E25F
:101E500087E9E82E83E0F82E8091040280FF0BC012
:101E600088811F928F93FF92EF920E941E060F901F
:101E70000F900F900F90115021961111EDCF80917E
:101E8000040280FF0AC085E993E0DF91CF911F91A2
:101E90000F91FF90EF900C948505DF91CF911F91EA
:101EA0000F91FF90EF900895E0918C01F0918D01DA
:101EB000309721F00480F581E02D09940895CF93A7
:101EC000DF93EC0180918A0190918B01C817D907AB
:101ED00009F1D0938B01C0938A01E0918C01F091BC
:101EE0008D013097B9F00680F781E02DCE0109957C
:101EF0008091040282FF0EC080FF0CC0DF93CF935D
:101F000087E893E09F938F930E941E060F900F9097
:101F10000F900F90DF91CF910895CF93DF93EC0155
:101F20008091880190918901C817D90709F1D09350
:101F30008901C0938801E0918C01F0918D01309767
:101F4000B9F00084F185E02DCE010995809104025D
:101F500082FF0EC080FF0CC0DF93CF9387E793E032
:101F60009F938F930E941E060F900F900F900F90DB
:101F7000DF91CF9108950C9481100E94F91B0C946D
:101F80002706CF92DF92EF92FF920F931F93CF938A
:101F9000DF9300D000D000D0CDB7DEB70E9450064E
:101FA0008FE8C82E81E0D82E00E010E0E02E802FD0
:101FB0000E942907F60141916F01F42EF826B1F431
:101FC0000F5F1F4F0031110589F78FEF89838A83D7
:101FD0001B820E94021C8160782F9D838C83498123
:101FE0005A816B818D810E94B61047C09091040286
:101FF00091FF04C08E830E9482108E8120E030E029
:102000004F2D50E0922FBA01022E02C075956795B0
:102010000A94E2F760FF2BC02983EA8221E030E0D6
:10202000690102C0CC0CDD1C9A95E2F790E08C218E
:102030009D21892B09F420E02B830E94021C8160E2
:10204000782F9D838C8349815A816B818D810E9479
:10205000B61049815A816B817C818D810E947C1BE5
:10206000F801E157FE4F8081C826C08206C02F5F6D
:102070003F4F2830310531F6A3CF0E947B1B0E94D1
:10208000EF1E10918E010E94FF0E181741F10E9461
:10209000FF0E80938E019091040292FF0EC090FF7C
:1020A0000CC01F928F9388EA93E09F938F930E94B6
:1020B0001E060F900F900F900F9080918E01269624
:1020C0000FB6F894DEBF0FBECDBFDF91CF911F9149
:1020D0000F91FF90EF90DF90CF900C948D1B269680
:1020E0000FB6F894DEBF0FBECDBFDF91CF911F9129
:1020F0000F91FF90EF90DF90CF9008950C943407EC
:1021000008950895EF92FF920F931F93CF93DF935B
:1021100081EC93E00E948505C0E0D0E08DE2E82EDE
:1021200081E0F82E03EB13E08C2F0E9429070E9418
:10213000651BFF92EF921F928F93DF93CF931F93B4
:102140000F930E941E0621968DB79EB708960FB674
:10215000F8949EBF0FBE8DBFC031D10529F7DF9126
:10216000CF911F910F91FF90EF900895CF93DF9340
:10217000CDB7DEB72B970FB6F894DEBF0FBECDBF3D
:10218000942F4F83252F588769877A878B874A85B5
:102190005B85452B21F02F3F09F59F3FF9F4DE01C8
:1021A000119686E0FD0111928A95E9F785E0FE011E
:1021B000379601900D928A95E1F749815A816B819A
:1021C0007C818D819E810E9491172B960FB6F89489
:1021D000DEBF0FBECDBFDF91CF9108954F815885EF
:1021E00069857A858B850E947C1BD9CFCF93882304
:1021F00009F465C0C82F8CEF8C0F813A20F080E580
:102200008C0F8E3248F48C2F0E943922811157C0D6
:102210008C2F0E941C1A0CC080E28C0F883058F45E
:10222000C77081E001C0880FCA95EAF70E94C71AFB
:10223000CF910C940B1B8BE58C0F833078F4C53A4F
:1022400029F0C63A31F083E890E005C081E890E0DB
:1022500002C082E890E0CF910C945F0F88E58C0F6C
:10226000853168F5C83A89F0C93A91F0CA3A99F0CF
:10227000CB3AA1F0CC3AA9F0CD3AB1F0CE3AB9F0D0
:10228000CF3AC1F080E090E017C082EE90E014C039
:1022900089EE90E011C08AEE90E00EC085EB90E0F0
:1022A0000BC086EB90E008C083EB90E005C084EBA8
:1022B00090E002C087EB90E0CF910C948D0FCF910E
:1022C0000895882349F19CEF980F913A20F090E50A
:1022D000980F9E3218F40E946F1A0DC090E2980F6A
:1022E000983058F4877091E001C0990F8A95EAF709
:1022F000892F0E94CD1A0C940B1B9BE5980F9330ED
:1023000020F480E090E00C945F0F885A853120F42F
:1023100080E090E00C948D0F0895882321F00E94B6
:10232000C71A0C940B1B0895882321F00E94CD1A24
:102330000C940B1B0895BF92CF92DF92EF92FF9205
:102340000F931F93CF93DF9300D000D000D0CDB771
:10235000DEB725E0FC01DE01119601900D922A9571
:10236000E1F7FC0140813181F280258122952F70B7
:1023700063817481672B09F4FEC23F3F19F44F3F1C
:1023800009F4F9C26C0149833A8389819A812E83C9
:102390000E94DB19182FB92E0E94DA190E94EA1840
:1023A000EB2DE295EF70F0E0E05AFF4F2E810C9498
:1023B000DF248B2D807F9B2D9F70092F882311F0A8
:1023C0000295007FFF2049F0002309F481C2802F8D
:1023D0000E94DA1A0E940B1B7BC2812F0E9461119E
:1023E000002309F4C8C2802F0E94E01A26960FB677
:1023F000F894DEBF0FBECDBFDF91CF911F910F913B
:10240000FF90EF90DF90CF90BF900C940B1B8B2D23
:10241000807F9B2D9F70092F803211F00295007FE5
:10242000112319F0113009F12AC0FF20B1F0802FDB
:10243000222351F1213041F526960FB6F894DEBFE4
:102440000FBECDBFDF91CF911F910F91FF90EF9005
:10245000DF90CF90BF900C94EA1A222319F021301C
:1024600009F489C20E94F31A2DC0FF20F1F0263032
:1024700008F081C20E94C41A802329F023C0FF20E3
:10248000F9F0211116C0802F26960FB6F894DEBF02
:102490000FBECDBFDF91CF911F910F91FF90EF90B5
:1024A000DF90CF90BF900C948D11253008F063C25F
:1024B00009C0F601858180FF0BC28F708583E3CF51
:1024C00021111BC2802F82C12B2D269526952370AA
:1024D00030E02115310521F021303105D1F04BC21A
:1024E000FF2021F0812F9B2D937002C080E090E0AF
:1024F00026960FB6F894DEBF0FBECDBFDF91CF9109
:102500001F910F91FF90EF90DF90CF90BF900C94B0
:102510005F0FFF2021F0812F9B2D937002C080E080
:1025200090E026960FB6F894DEBF0FBECDBFDF91C8
:10253000CF911F910F91FF90EF90DF90CF90BF90C0
:102540000C948D0F812FFF2019F00E94751D02C081
:102550000E94DD1D26960FB6F894DEBF0FBECDBFDC
:10256000DF91CF911F910F91FF90EF90DF90CF906F
:10257000BF900C94621E8B2D837009F07BC0F1100C
:10258000FAC1812F829586958770880F880F912FC9
:102590009F70C92ED12CE12CF12C082E04C0CC0C3C
:1025A000DD1CEE1CFF1C0A94D2F714FF12C04FE092
:1025B00050E060E070E004C0440F551F661F771FB5
:1025C0008A95D2F7CB01BA01609570958095909568
:1025D00003C060E070E0CB012B2D2695269523707B
:1025E000422F50E042305105D9F04330510569F196
:1025F0006C297D298E299F294130510551F126965C
:102600000FB6F894DEBF0FBECDBFDF91CF911F9103
:102610000F91FF90EF90DF90CF90BF900C94FF1838
:102620006C297D298E299F2926960FB6F894DEBF46
:102630000FBECDBFDF91CF911F910F91FF90EF9013
:10264000DF90CF90BF900C9411190E94FF18C70122
:10265000B60126960FB6F894DEBF0FBECDBFDF9150
:10266000CF911F910F91FF90EF90DF90CF90BF908F
:102670000C94ED18FF2019F08B2D817001C0869508
:10268000882309F478C1812F829586958770880FF9
:10269000880F912F9F70C92ED12CE12CF12C082E80
:1026A00004C0CC0CDD1CEE1CFF1C0A94D2F714FFF6
:1026B00012C04FE050E060E070E004C0440F551FCE
:1026C000661F771F8A95D2F7CB01BA016095709586
:1026D0008095909503C060E070E0CB012B2D26958E
:1026E00026952370422F50E042305105D9F04330F7
:1026F000510569F16C297D298E299F2941305105A9
:1027000051F126960FB6F894DEBF0FBECDBFDF9114
:10271000CF911F910F91FF90EF90DF90CF90BF90DE
:102720000C94B6196C297D298E299F2926960FB6FF
:10273000F894DEBF0FBECDBFDF91CF911F910F91F7
:10274000FF90EF90DF90CF90BF900C94C8190E943B
:10275000B619C701B60126960FB6F894DEBF0FBEB4
:10276000CDBFDF91CF911F910F91FF90EF90DF9040
:10277000CF90BF900C94A419103FC9F128F480E4C5
:10278000810F803250F09FC0123F09F461C008F4FD
:102790004AC0133F09F471C096C0012F00718B2D00
:1027A0008F71FF2051F00E943D19812F002319F0F5
:1027B0008295807F69CE8F7067CE0E945E19812FCF
:1027C000002319F08295807F01C08F7026960FB686
:1027D000F894DEBF0FBECDBFDF91CF911F910F9157
:1027E000FF90EF90DF90CF90BF900C949411FF205A
:1027F000B1F0253008F0BFC08B2D8F7126960FB633
:10280000F894DEBF0FBECDBFDF91CF911F910F9126
:10281000FF90EF90DF90CF90BF900C9483192630FB
:1028200008F0A9C0E9CFFF20A9F08B2D8F71269663
:102830000FB6F894DEBF0FBECDBFDF91CF911F91D1
:102840000F91FF90EF90DF90CF90BF900C943D19C7
:10285000FF2059F38B2D8F7126960FB6F894DEBFAB
:102860000FBECDBFDF91CF911F910F91FF90EF90E1
:10287000DF90CF90BF900C945E19FF2099F08B2DC4
:102880008F7126960FB6F894DEBF0FBECDBFDF91D5
:10289000CF911F910F91FF90EF90DF90CF90BF905D
:1028A0000C94281926960FB6F894DEBF0FBECDBF44
:1028B000DF91CF911F910F91FF90EF90DF90CF901C
:1028C000BF900C942319FF20A9F0222309F4ADCF67
:1028D000812F26960FB6F894DEBF0FBECDBFDF91D5
:1028E000CF911F910F91FF90EF90DF90CF90BF900D
:1028F0000C94F610222309F4ADCF812F26960FB643
:10290000F894DEBF0FBECDBFDF91CF911F910F9125
:10291000FF90EF90DF90CF90BF900C9461114B2D02
:102920004F70612FC6010E94EF1C26960FB6F894D7
:10293000DEBF0FBECDBFDF91CF911F910F91FF90F2
:10294000EF90DF90CF90BF900C9435184B2D4F70C7
:10295000612FC60126960FB6F894DEBF0FBECDBF1D
:10296000DF91CF911F910F91FF90EF90DF90CF906B
:10297000BF900C94F21C26960FB6F894DEBF0FBEE3
:10298000CDBFDF91CF911F910F91FF90EF90DF901E
:10299000CF90BF9008950E94E71A0E94B61A0E9435
:1029A0000B1B0E94941F0E94621E80E090E00E9418
:1029B0005F0F80E090E00C948D0F0E94D71A0C946A
:1029C000CB140E94DB19292F22952F7030E02C3078
:1029D00031054CF42A303105C4F42250310922303B
:1029E000310540F023C02C303105D1F02F303105B6
:1029F000B9F01CC0853A28F48430B0F4823028F451
:102A000013C090E2980F983078F0883E30F4803E02
:102A100058F48450813A50F407C0803F39F404C020
:102A200093FB882780F9089581E0089580E0089558
:102A3000CF93DF9300D000D01F92CDB7DEB70F90B9
:102A40000F900F900F900F90DF91CF910895CF933B
:102A5000DF9300D000D000D0CDB7DEB726960FB6FA
:102A6000F894DEBF0FBECDBFDF91CF9108951F93C5
:102A7000CF93DF93C0919F0116E08091A001C8170A
:102A800099F0D0E01C9FF0011D9FF00D1124EF552F
:102A9000FE4F4081518162817381848195810E94C2
:102AA00027152196C770E9CFDF91CF911F91089527
:102AB0004091D1015091D2016091D3017091D40124
:102AC0008091D5019091D6010C9427158091D60163
:102AD00082958F7009F054C08091D301882309F446
:102AE0004FC080919F01A091A0016091D101709190
:102AF000D2014091D4015091D501B6E08A1709F472
:102B00003FC090E041155105C1F17F3F11F46F3F87
:102B1000A1F1B89FF001B99FF00D1124EF55FE4FC0
:102B2000218172132AC02081621327C022812111C2
:102B300024C0238134812417350710F42150310932
:102B4000241B350B2C323140C0F42091D6012F705C
:102B500020612093D60126E0289FF001299FF00DE7
:102B60001124EA55FE4F80818F708061808381ED52
:102B700091E00E949B110C94371501968770BECF8F
:102B80000895CF92DF92EF92FF920F931F93CF930E
:102B9000DF93CDB7DEB762970FB6F894DEBF0FBEF6
:102BA000CDBF8C0185E0F801DE011D9601900D92EC
:102BB0008A95E1F7D8014C9111965C911197129684
:102BC0006C9112971396CD90DC9014973091D101AF
:102BD0007091D2018091D4019091D501009709F4B0
:102BE00073C17F3F19F43F3F09F46EC1E090D301F8
:102BF000EE2009F4C5C02091D601C816D90650F0C0
:102C0000F601E81BF90BCF01FF24F3948C329140BD
:102C1000C8F009C0809590958C0D9D1DFF24F394FC
:102C20008C32914078F0F12C207F09F0C6C07C2DC9
:102C3000D98AC88A89890E94181581ED91E00E947D
:102C40009B11B1C0822F807F09F045C0751313C05E
:102C5000341311C061110FC02F7020612093D60171
:102C60000E94581581ED91E00E949B118091D60140
:102C7000F80185832EC0CD2819F15F3F11F44F3F35
:102C8000F9F0F62E61111CC080919F012091A001E6
:102C900036E0821709F45BC090E0389FF001399F5D
:102CA000F00D1124EF55FE4F7181571306C070814E
:102CB000471303C07281711103C001968770E9CF79
:102CC000F62E662309F41DC18091D60181608093A0
:102CD000D601F12C16C1751309C0341307C0611158
:102CE00005C08091D601F8018583C8C04D875E87F5
:102CF0008D859E856A8B0E94E1146A898823E1F1A3
:102D00006623D1F12091D601822F82958F7090E0B9
:102D1000029774F08091D1019091D20198878F83AE
:102D20001986DB86CA862C87CE0107960E949B11E6
:102D300086E0F801A1EDB1E001900D928A95E1F7EE
:102D40000E9466150E945815FF24F394DAC04D873F
:102D50005E878D859E850E94DB19292F22952F7015
:102D600030E0223031050CF0BFC09F7009F0B9C0CF
:102D7000805E883008F4C5C0C8010E949B11E4CF72
:102D8000C816D90608F453C0F601E81BF90BCF01A9
:102D90008C32914008F453C0F12C7C2DD98AC88A1A
:102DA00089890E941815E1EDF1E086E0DF011D92AE
:102DB0008A95E9F70E945815A4C0751314C03413FE
:102DC00012C0611110C08091D601F8018583C8013D
:102DD0000E949B1186E0E1EDF1E0DF011D928A95F2
:102DE000E9F7FE2C8EC04D875E878D859E856A8BA8
:102DF0000E94E1146A89882309F4BECF662309F48E
:102E0000BBCF2091D601822F82958F7090E00297E0
:102E10000CF48ECF8091D1019091D2019A83898355
:102E20001B82DD82CC822E83CE0101967FCF8095DE
:102E300090958C0D9D1D8C32914008F0ADCFF62EF3
:102E4000662309F499CF75132EC034132CC020913A
:102E5000D60120FD1FC0822F82958F70D9F0D80136
:102E600015962C9315978F3049F08F5F982F929578
:102E7000907F822F8F70892B15968C93C8010E94AA
:102E80009B1186E0F801A1EDB1E001900D928A95C9
:102E9000E1F790CF86E0F801A1EDB1E001900D924D
:102EA0008A95E1F72EC04D875E878D859E850E94AD
:102EB000E11481113DCF8091D60181608093D601CC
:102EC000C8010E949B111DC0662309F455CF4D8790
:102ED0005E878D859E850E94E114882309F44CCF7E
:102EE00027CF811145CF0DC0243031050CF044CFE0
:102EF0009F7009F43DCFD80115969C91907F09F001
:102F000037CF8F2D62960FB6F894DEBF0FBECDBFC0
:102F1000DF91CF911F910F91FF90EF90DF90CF90B5
:102F200008951F93CF93DF93CDB7DEB72C970FB6DD
:102F3000F894DEBF0FBECDBF4F83588769877A876D
:102F40008B879C87CE0107960E94C115882369F064
:102F50008F8198852A853B85232BF1F19F3F09F0CE
:102F600063C08F3F09F060C037C086E0FE0137962E
:102F7000DE01119601900D928A95E1F76F817885B7
:102F8000EA85FB85309741F17F3F11F46F3F21F1D6
:102F90002091A00130E0C9010196877099274091E6
:102FA0009F0150E08417950709F447C069837A832D
:102FB000FD83EC8396E0929FD001939FB00D112486
:102FC000AF55BE4FFE01319601900D929A95E1F7F3
:102FD0008093A0010E94371516E080919F01909187
:102FE000A0018917C1F1189FC00111248F559E4F70
:102FF0000E94C115882379F1E0919F011E9FF00185
:103000001124EF55FE4F408151816281738184818B
:1030100095810E94271580919F0190E0019687700D
:10302000992780939F01D9CF4F81588569857A85EB
:103030008B859C850E942715CFCF0E94DD141092AE
:10304000A00110929F01E1EDF1E086E0DF011D9209
:103050008A95E9F7C1CF2C960FB6F894DEBF0FBE64
:10306000CDBFDF91CF911F910895DF92EF92FF9234
:103070000F931F93CF93DF93FC01892B09F48AC030
:10308000E12CF12CDD24D394EF0121968491853736
:1030900009F461C058F4843708F04EC0843008F059
:1030A0006AC08130D1F0823071F174C0883709F480
:1030B0005DC050F4863709F455C0873709F06AC0FF
:1030C0008E2D0E94D41A54C09CE7980F903708F0B8
:1030D00061C08F770E94611150C08F010E5F1F4F3A
:1030E000FE01849190E2980F983050F48770FD2D86
:1030F00001C0FF0F8A95EAF78F2F0E94DA1A14C0D9
:103100000E94F61013C08F010E5F1F4FFE01C49185
:1031100080E28C0F883060F4C7708D2D01C0880F5D
:10312000CA95EAF70E94E01A0E940B1BE80125C02D
:103130008C2F0E946111FACF9F012E5F3F4FFE013D
:10314000C491CC2369F08FE99FE00197F1F700C0AB
:103150000000C150F6CF9F012E5F3F4FFE01F4905B
:10316000E9010BC00E94C41AE82E07C00E94D71ABA
:103170000E940B1B02C00E94F6108F2D882341F085
:10318000EFE9FFE03197F1F700C000008150F6CF82
:10319000FE017ACFDF91CF911F910F91FF90EF90B9
:1031A000DF9008956093DB017093DC018093DD0173
:1031B0009093DE010E948B1B0C94CB146093D7017B
:1031C0007093D8018093D9019093DA010E948C1BEF
:1031D0000C94CB1408950C94D2180F931F93009164
:1031E000DB011091DC012091DD013091DE01602BCB
:1031F000712B822B932B1F910F910C94D2180F934C
:103200001F930091DB011091DC012091DD013091D1
:10321000DE0160237123822393231F910F910C946D
:10322000D2180F931F930091DB011091DC012091C4
:10323000DD013091DE0160277127822793271F91DE
:103240000F910C94D21860E070E0CB010C94DE1862
:103250000F931F9341E050E060E070E08A019B0112
:1032600004C0000F111F221F331F8A95D2F7C90116
:10327000B8011F910F910C94DE180F931F9341E03A
:1032800050E060E070E004C0440F551F661F771FD8
:103290008A95D2F78091D7019091D801A091D90158
:1032A000B091DA018A019B01082B192B2A2B3B2BA9
:1032B000C901B8011F910F910C94DE180F931F9351
:1032C00041E050E060E070E004C0440F551F661F0D
:1032D000771F8A95D2F740955095609570958091AB
:1032E000D7019091D801A091D901B091DA018A015A
:1032F0009B01082319232A233B23C901B8011F91ED
:103300000F910C94DE180F931F9341E050E060E0A2
:1033100070E004C0440F551F661F771F8A95D2F7CF
:103320008091D7019091D801A091D901B091DA0193
:103330008A019B01082719272A273B27C901B801C1
:103340001F910F910C94DE180F931F930091D701DA
:103350001091D8012091D9013091DA01602B712BA5
:10336000822B932B1F910F910C94DE180F931F93B8
:103370000091D7011091D8012091D9013091DA0143
:1033800060237123822393231F910F910C94DE18E5
:103390000F931F930091D7011091D8012091D9016B
:1033A0003091DA0160277127822793271F910F91AF
:1033B0000C94DE180895CF92DF92EF92FF920F9354
:1033C0001F93CF93DF938C01C090DB01D090DC0181
:1033D000E090DD01F090DE014091D7015091D801DD
:1033E0006091D9017091DA01C42AD52AE62AF72A18
:1033F000CFE1D0E0D701C6010C2E04C0B695A79549
:10340000979587950A94D2F780FF07C0B8018C2F53
:103410000E94C51C8130910531F4219758F7B801FD
:1034200080E00E94C51CDF91CF911F910F91FF900A
:10343000EF90DF90CF90089590910A01992321F0A9
:1034400090910B01911109C020910C0130910D0157
:10345000F90132969FEF40E030C0982F96959695EF
:1034600096959F31A0F4E0910C01F0910D01E90FC8
:10347000F11D877021E030E0A90102C0440F551F03
:103480008A95E2F7CA019181892B818308959091F1
:10349000040290FF23C01F928F938DEE93E09F93C1
:1034A0008F930E941E060F900F900F900F9008951B
:1034B0009F3F39F04F5F4E3141F051915813F8CF93
:1034C0000DC05111F7CF942FF5CF9F3F39F0F9017F
:1034D000E90FF11D97FDFA95828308950895909163
:1034E0000A01992321F090910B01911109C02091BB
:1034F0000C0130910D01F9013296205E3F4F30C032
:10350000982F9695969596959F31A8F4E0910C0189
:10351000F0910D01E90FF11D877021E030E0A90164
:1035200002C0440F551F8A95E2F7CA018095918128
:103530008923818308959091040290FF16C01F9201
:103540008F938FEC93E09F938F930E941E060F90B2
:103550000F900F900F9008953196E217F30729F01E
:1035600090819813F9CF1082F7CF089581E090E011
:10357000E0910C01F0910D01E80FF91F1082019606
:1035800080329105A9F708958091030208959091E2
:103590000302892B80930302089580959091030282
:1035A0008923809303020895809303020895109263
:1035B0000302089590910202892B809302020895DC
:1035C00080959091020289238093020208951092BF
:1035D000020208958093E1010E94021C9093E00191
:1035E0008093DF0108951092E1011092E0011092A2
:1035F000DF01089580910C0190910D01FC0131963D
:103600009C01205E3F4F80E0919191118F5FE21706
:10361000F307D1F70895E0910C01F0910D0180912D
:1036200003028083E0910C01F0910D019081809163
:103630000202892B80838091E1018823D9F10E94C5
:10364000021C2091DF013091E0018217930748F0BE
:103650000E94021C2091DF013091E001821B930B3C
:103660000AC00E94021C2091DF013091E0012095E8
:103670003095820F931F8C32914070F0809104023C
:1036800080FF08C08BE094E09F938F930E941E06FA
:103690000F900F900E94F31AE0910C01F0910D0130
:1036A00090818091E101892B80830E94FA1A811117
:1036B0000E94F31A80910C0190910D010C940B0F54
:1036C000909339018093380108958295982F9C7CBE
:1036D000392F36953695282F237344E0249FC00157
:1036E0001124932F982B292F2A7A2695892F8575B7
:1036F000880F822B08950895CF93DF9300D000D0D8
:103700001F92CDB7DEB70F900F900F900F900F90D4
:10371000DF91CF910895089508950C947E108091C3
:103720001902843021F11092050220E488E190E032
:103730000FB6F894A895809360000FBE20936000A8
:1037400083B7817F846083BF83B7816083BF7894B0
:10375000889583B78E7F83BF0FB6F894A895809124
:103760006000886180936000109260000FBE089531
:10377000CF930E9432070E9450060E943307C0E098
:103780008C2F0E942907811104C0CF5FC031C1F77F
:1037900001C081E0CF9108950E9480100C94DD1447
:1037A0001F920F920FB60F9211248F939F93AF9396
:1037B000BF9380910502811113C080910602909100
:1037C0000702A0910802B09109024196A11DB11D06
:1037D0008093060290930702A0930802B093090217
:1037E000BF91AF919F918F910F900FBE0F901F903F
:1037F000189582E084BD93E095BD9AEF97BD8093C4
:103800006E0008952FB7F8948091060290910702F8
:10381000A0910802B09109022FBF08952FB7F89424
:10382000609106027091070280910802909109024E
:103830002FBF0895CF92DF92EF92FF920F931F93C5
:103840002FB7F89440910602509107026091080248
:10385000709109022FBF6A017B01EE24FF248C01C5
:1038600020E030E0C016D106E206F30610F4415025
:1038700051099A01281B390BC9011F910F91FF9023
:10388000EF90DF90CF900895CF92DF92EF92FF926A
:103890000F931F932FB7F894C0900602D0900702A1
:1038A000E0900802F09009022FBF97018601061BE5
:1038B000170B280B390BC616D706E806F90618F0C1
:1038C000C901B80106C0C901B80161507109810977
:1038D00091091F910F91FF90EF90DF90CF90089585
:1038E0001F920F920FB60F9211248F939F93AF9355
:1038F000BF938091060290910702A0910802B091B7
:1039000009020196A11DB11D809306029093070242
:10391000A0930802B0930902BF91AF919F918F913C
:103920000F900FBE0F901F9018950E94180CF894DE
:103930002FEF87EA91E6215080409040E1F700C0E8
:10394000000087E090EBDC01809322029093230239
:10395000A0932402B09325029CE088E10FB6F8946E
:10396000A895809360000FBE90936000FFCF28E081
:10397000929FF0011124E80FF11DE052FF4F949146
:10398000892F8F7092959F700895CF93C82FCB0188
:103990000E94B71C282F30E080E1989FA0011124DD
:1039A000422B532B4038510519F480E090E015C0AC
:1039B0009770E92FF0E088E0C89FE00DF11D112419
:1039C00084E0EE0FFF1F8A95E1F7E20FF31FEE0F81
:1039D000FF1FE050F84985919491CF91089580E0C0
:1039E00090E00895089580910C0280FF0BC06091D3
:1039F000110185E0689FB001112475956795759553
:103A000067952BC081FF09C06091110185E0689F17
:103A1000B00111247595679520C082FF07C06091A1
:103A2000110185E0689FB001112417C090910D022B
:103A30009923D1F060911001961788F72091110118
:103A400085E0289F90011124929FA001939F500D23
:103A5000112470E0CA010E94CB246038710540F443
:103A60006115710539F002C065E070E0862F089598
:103A70008FE7089581E0089580910C0280FF08C0CF
:103A800060910F0170E0759567957595679521C0F8
:103A900081FF06C060910F0170E07595679519C0B0
:103AA00082FF04C060910F0170E010C090910D0280
:103AB0009923C1F060910E019617A0F780910F0134
:103AC000899FC001112470E00E94CB2460387105E9
:103AD00028F46115710521F0862F08958FE7089568
:103AE00081E0089561E070E0F4CF803F21F40E940E
:103AF000F31C819504C0813F29F40E94F31C80933C
:103B000010020895823F21F40E94F31C819504C0A5
:103B1000833F29F40E94F31C80930F020895893F8C
:103B200019F40E943C1D05C08A3F31F40E943C1DDF
:103B300081958093110208958B3F21F40E943C1DD2
:103B4000819504C08C3F29F40E943C1D8093120291
:103B50000895843F21F480910E02816017C0853F53
:103B600021F480910E02826011C0863F21F4809181
:103B70000E0284600BC0873F21F480910E028860A2
:103B800005C0883F31F480910E02806180930E025F
:103B900008958D3F21F480910C0281600BC08E3F0F
:103BA00021F480910C02826005C08F3F29F480913E
:103BB0000C02846080930C020895803F39F4809158
:103BC000100287FF6CC01092100269C0813F29F477
:103BD000809110021816BCF362C090910F02823FD0
:103BE00029F497FF5CC010920F0259C0833F19F46B
:103BF0001916CCF354C0893F41F480911102181674
:103C00000CF04DC0109211024AC08A3F29F48091F5
:103C1000110287FF44C0F6CF8B3F39F48091120226
:103C200087FF3DC0109212023AC08C3F29F4809168
:103C300012021816BCF333C0843F21F480910E02A7
:103C40008E7F17C0853F21F480910E028D7F11C0B9
:103C5000863F21F480910E028B7F0BC0873F21F4B9
:103C600080910E02877F05C0883F31F480910E025B
:103C70008F7E80930E0213C08D3F21F480910C0241
:103C80008E7F0BC08E3F21F480910C028D7F05C08A
:103C90008F3F29F480910C028B7F80930C028091DE
:103CA0000F0281110EC08091100281110AC0809113
:103CB0001102811106C080911202811102C010927E
:103CC0000D0208958091040283FF7EC084E494E095
:103CD0000E94850580910E021F928F938FE394E0DE
:103CE0009F938F930E941E068DE394E00E948505AA
:103CF00080910F02282F082E000C330B3F938F93D7
:103D00008AE394E09F938F930E941E0688E394E0D9
:103D10000E94850580911002282F082E000C330B7D
:103D20003F938F9385E394E09F938F930E941E06A9
:103D300083E394E00E94850580911102282F082ECC
:103D4000000C330B3F938F9380E394E09F938F930A
:103D50000E941E068EE294E00E9485058091120268
:103D6000282F082E000C330B3F938F938BE294E0A7
:103D70009F938F930E941E0688E294E00E9485051F
:103D800080910D021F928F9385E294E09F938F9311
:103D90000E941E0683E294E00E94850580910C0239
:103DA0001F928F9380E294E09F938F930E941E0650
:103DB0008DE194E00E9485058DB79EB74C960FB6B5
:103DC000F8949EBF0FBE8DBF8EE092E00E94540F0C
:103DD0000E94021C90930B0280930A0208951F9385
:103DE000CF93DF9380910A0290910B020E941A1CDC
:103DF000AC0190910D02992321F02091120130E045
:103E000006C0209113018AE0289F900111244217D7
:103E1000530708F485C080910F02C0911002D09121
:103E2000110210911202811107C0C11175C0D11188
:103E300073C0111171C074C09F3F19F09F5F9093C0
:103E40000D02181624F40E94F31C80930F02809137
:103E50000F0287FF05C00E94F31C819580930F021B
:103E60001C1624F40E94F31C80931002809110020F
:103E700087FF05C00E94F31C81958093100260911A
:103E80000F02662331F1C0911002CC2311F1062EEE
:103E9000000C770B880B990B0E94C62323E333E3B6
:103EA00043E35FE30E942A240E948E2360930F0263
:103EB0006C2FCC0F770B880B990B0E94C62323E342
:103EC00033E343E35FE30E942A240E948E2360933E
:103ED00010021D1624F40E943C1D80931102809153
:103EE000110287FF05C00E943C1D8195809311023D
:103EF000111624F40E943C1D80931202809112023C
:103F000087FF05C00E943C1D819580931202DF91BE
:103F1000CF911F910C94621E9F3F09F08FCF97CFD6
:103F2000DF91CF911F910895EEE0F2E085E0DF018F
:103F30001D928A95E9F710920D0210920C020895D5
:103F400087E696E00E9485051F9281E08F931F927D
:103F500085E08F9389E196E09F938F930E941E06E0
:103F60000F900F900F900F900F900F900895833047
:103F7000E9F128F4813061F0823009F1089585304B
:103F800009F462C008F449C0863009F474C0089589
:103F900080911301262F30E0280F311D2F3F31056E
:103FA00024F4680F6093130103C08FEF8093130113
:103FB000809113011F928F9382E595E072C08091EA
:103FC0001201262F30E0280F311D2F3F310524F438
:103FD000680F6093120103C08FEF809312018091EC
:103FE00012011F928F9380E495E05BC080911101D4
:103FF000262F30E0280F311D2F3F310524F4680FA4
:104000006093110103C08FEF809311018091110122
:104010001F928F938DE295E044C080911001262F6E
:1040200030E0280F311D2F3F310524F4680F6093D5
:10403000100103C08FEF80931001809110011F9237
:104040008F9388E195E02DC080910F01262F30E0FD
:10405000280F311D2F3F310524F4680F60930F01A5
:1040600003C08FEF80930F0180910F011F928F93F8
:104070008FEF94E016C080910E01262F30E0280FBC
:10408000311D2F3F310524F4680F60930E0103C0EA
:104090008FEF80930E0180910E011F928F9384EE1B
:1040A00094E09F938F930E941E060F900F900F90A5
:1040B0000F900895833081F128F4813059F08230D7
:1040C000D1F00895853009F449C0B8F1863009F47B
:1040D00056C0089580911301681720F4861B8093C1
:1040E000130102C010921301809113011F928F934C
:1040F00085ED94E054C080911201681720F4861B6E
:104100008093120102C010921201809112011F923D
:104110008F9383EC94E043C080911101681720F4E1
:10412000861B8093110102C0109211018091110130
:104130001F928F9380EB94E032C08091100168173A
:1041400020F4861B8093100102C010921001809110
:1041500010011F928F938BE994E021C080910F0191
:10416000681720F4861B80930F0102C010920F0184
:1041700080910F011F928F9382E894E010C080918C
:104180000E01681720F4861B80930E0102C0109266
:104190000E0180910E011F928F9387E694E09F930A
:1041A0008F930E941E060F900F900F900F9008950E
:1041B000CF93C82F1F928F938CE697E09F938F9396
:1041C0000E941E0681E090E0A0E0B0E0BC01CD01BD
:1041D00004C0660F771F881F991FCA95D2F70E94E7
:1041E000EB180F900F900F900F90CF910C94DD145F
:1041F000CF938732A8F58E3108F02BC1803109F4B6
:104200009FC0F8F4873009F464C0A8F4863009F040
:1042100024C180910402817F8E7F8093040281E714
:1042200097E00E9485058BE59AE00E94850581E074
:10423000809314024CC08B30F1F18E3009F46CC0C5
:104240000CC1863109F4B0C020F4813109F4EDC00D
:1042500004C1893109F491C08B3109F449C0FDC012
:10426000883349F150F4893209F4F1C0853309F4F7
:10427000EEC0873209F0F1C0EAC0833409F4E7C028
:1042800028F48A3308F4E9C08953E4C0883409F07B
:10429000E4C00E94DD148AE49AE00E9485052FEFB5
:1042A00083ED90E3215080409040E1F700C0000092
:1042B0000E94951C0CC088E997E05CC081E39AE0FD
:1042C0000E94850580910402816080930402C1E010
:1042D000C9C080910402C82FC17080FFEFCF8DE369
:1042E0009AE00E94850580910402817F8E7F3DC007
:1042F0009091040291FBCC27C0F981E0C827892F57
:10430000C0FB81F980930402CC2319F084E29AE087
:1043100027C086E19AE02EC09091040292FBCC2740
:10432000C0F981E0C827892FC0FB82F9809304027D
:10433000CC2319F087E09AE013C087EF99E01AC008
:104340009091040293FBCC27C0F981E0C827892F04
:10435000C0FB83F980930402CC2351F08BEE99E0EB
:104360000E948505809104028160809304027AC0D6
:104370008EED99E00E948505AACF8FEC99E00E940E
:10438000850582EA99E00E9485058BE699E00E9406
:1043900085058EE399E00E94850584EF98E00E94F0
:1043A000850586EC98E0E6CF88EB98E00E948505CD
:1043B0000E94FF0E1F928F938EE998E09F938F9338
:1043C0000E941E0680910A011F928F9387E898E051
:1043D0009F938F930E941E06809187011F928F9357
:1043E00084E798E09F938F930E941E0680910B01B3
:1043F0001F928F9381E698E09F938F930E941E06F1
:104400000E940E1C9F938F937F936F938AE498E092
:104410009F938F930E941E068DB79EB746960FB648
:10442000F8949EBF0FBE8DBF52CF0E94DD14C09185
:104430000B0181E0C827C0930B01CC2329F080E455
:1044400098E00E9485050EC085E398E093CF80E058
:1044500001C08D510E94D8203ACF83E398E00E949A
:104460008505C0E08C2FCF91089580E0089580E00D
:104470000895CF93C82F80911402813071F020F0FD
:10448000823009F44BC042C1E0910C01F0910D0162
:104490008081823209F03CC107C0E0910C01F091AB
:1044A0000D018081823261F48C2F0E9435228111AE
:1044B00004C08C2F0E94F8202FC081E090E02CC017
:1044C0008C2F0E943722811126C0C431E1F070F494
:1044D000CB3081F0C031D1F40E94A01F84E697E078
:1044E0000E94850582E08093140215C0C93259F0FC
:1044F000C83361F481E797E00E94850588E697E07C
:104500000E94850508C01092140204C182E697E05B
:104510000E948505FFC081E08170FEC0C43228F58D
:10452000CE3108F0C1C0CB30A1F1D0F4C73009F0D2
:10453000D3C08EE18093130182E3809312018AE05D
:104540008093110184E18093100188E080930F0132
:1045500088E280930E0188E096E00E948505BFC046
:10456000C33149F1C431C1F0B7C0CB3409F4A9C09B
:1045700028F4C93289F0C83361F0AEC0C13509F4FE
:104580009EC0C23509F499C0CE3409F0A5C06AE0D6
:104590009EC00E94A01FA3C080911302882319F01F
:1045A000109213029CC085E196E00E94850581E08F
:1045B00080931402B1C08FEE95E00E9485058DEDC9
:1045C00095E00E948505809113011F928F938AEDDB
:1045D00095E09F938F930E941E0688ED95E00E94C0
:1045E000850586EC95E00E948505809112011F9259
:1045F0008F9383EC95E09F938F930E941E0681EC2E
:1046000095E00E94850582EB95E00E9485058091EA
:1046100011011F928F938FEA95E09F938F930E94D1
:104620001E068DEA95E00E9485058CE995E00E94C2
:104630008505809110011F928F9389E995E09F93E2
:104640008F930E941E0687E995E00E94850582E807
:1046500095E00E94850580910F011F928F938FE74F
:1046600095E09F938F930E941E068DE795E00E9430
:10467000850586E695E00E94850580910E011F92D2
:104680008F9383E695E09F938F930E941E0681E6A9
:1046900095E00E9485058DB79EB748960FB6F894B1
:1046A0009EBF0FBE8DBF1BC0CE51EC2FF0E0E25D70
:1046B000FE4F80818093130212C061E003C061E06D
:1046C00006C06AE0809113020E94B71F08C0809163
:1046D00013020E945A2003C086E096E013C0809126
:1046E0001302882369F01F928F9380E096E09F93D6
:1046F0008F930E941E060F900F900F900F9004C092
:104700008DEF95E00E94850581E006C010921402AD
:1047100080E002C080E000CFCF9108950E949523F1
:104720006894B1110C94242408950E94092488F0FF
:104730009F5798F0B92F9927B751B0F0E1F0660F65
:10474000771F881F991F1AF0BA95C9F714C0B130A6
:1047500091F00E942324B1E008950C942324672F44
:10476000782F8827B85F39F0B93FCCF386957795D5
:104770006795B395D9F73EF49095809570956195BE
:104780007F4F8F4F9F4F0895E89409C097FB3EF4E9
:1047900090958095709561957F4F8F4F9F4F99238E
:1047A000A9F0F92F96E9BB279395F695879577950C
:1047B0006795B795F111F8CFFAF4BB0F11F460FFCC
:1047C0001BC06F5F7F4F8F4F9F4F16C0882311F024
:1047D00096E911C0772321F09EE8872F762F05C038
:1047E000662371F096E8862F70E060E02AF09A95D3
:1047F000660F771F881FDAF7880F9695879597F9C8
:10480000089557FD9058440F551F59F05F3F71F0C0
:104810004795880F97FB991F61F09F3F79F0879527
:104820000895121613061406551FF2CF4695F1DFB0
:1048300008C0161617061806991FF1CF8695710540
:10484000610508940895E894BB2766277727CB0174
:1048500097F908950E943D240C94AE240E94A02450
:1048600038F00E94A72420F0952311F00C9497248F
:104870000C949D2411240C9424240E94012470F390
:10488000959FC1F3950F50E0551F629FF001729FF5
:10489000BB27F00DB11D639FAA27F00DB11DAA1F04
:1048A000649F6627B00DA11D661F829F2227B00D51
:1048B000A11D621F739FB00DA11D621F839FA00DDC
:1048C000611D221F749F3327A00D611D231F849F2C
:1048D000600D211D822F762F6A2F11249F57504083
:1048E0009AF0F1F088234AF0EE0FFF1FBB1F661FFE
:1048F000771F881F91505040A9F79E3F510580F0C7
:104900000C9497240C9424245F3FE4F3983ED4F352
:10491000869577956795B795F795E7959F5FC1F76A
:10492000FE2B880F911D9695879597F9089597F915
:104930009F6780E870E060E008959FEF80EC089545
:1049400000240A941616170618060906089500246E
:104950000A9412161306140605060895092E0394E8
:10496000000C11F4882352F0BB0F40F4BF2B11F45C
:1049700060FF04C06F5F7F4F8F4F9F4F0895991B5B
:1049800079E004C0991F961708F0961B881F7A9546
:10499000C9F78095089597FB072E16F4009407D069
:1049A00077FD09D00E94E52407FC05D03EF49095E0
:1049B00081959F4F0895709561957F4F0895EE0FF3
:1049C000FF1F0590F491E02D0994AA1BBB1B51E138
:1049D00007C0AA1FBB1FA617B70710F0A61BB70B6F
:1049E000881F991F5A95A9F780959095BC01CD0114
:0649F0000895F894FFCFCA
:1049F6003B072C080908D507A1070101E201280891
:104A0600140A321E404D3622393703EA02B40292A6
:104A1600025902CC01E501FE01170237020001022C
:084A260003040506070809005E
:1068000088000000000000000400050006000700EA
:10681000080009000A000B000C000D000E000F001C
:1068200010001100120013001400150016001700CC
:10683000180019001A001B001C001D001E001F007C
:10684000200021002200230024002500260027002C
:10685000280035002A002B002C002D002E002F00D0
:1068600030000000320033003400290036003700C9
:106870003800E00000000000000000000000000000
:106880000000000000000000000000000000000008
:1068900000000000000000000000000000004F00A9
:1068A00050005100520000000000000000000000F5
:1068B00000000000000000000000000000000000D8
:1068C00000000000000000000000000000000000C8
:1068D00000000000000000000000000000000000B8
:1068E0000000000000000000890087008A008B0083
:1068F000F1A1E100E200E300F1A1E500E600000003
:106900000100000000000000EA4401000100E24430
:106910000100010001005500460054004A004B00F0
:10692000560057004700480001000100E9440100FB
:106930000100010001000100010001003A003B00DC
:106940003C003D003E003F0040004100420043004B
:10695000580001004C00390001004400450052007D
:1069600001000000010050004F0081404D004E002A
:1069700051000100000000000000000000000000C5
:106980000000000000000000000000000000000007
:1069900000000000000000000000000000004D00AA
:1069A0004A004E004B000000000000000000000004
:1069B00000000000000000000000000000000000D7
:1069C00000000000000000000000000000000000C7
:1069D00000000000000000000000000000000000B7
:1069E000000000000000000049000100010001005B
:1069F0000100010001000100010001000100000090
:00000001FF
